:100000000C9434000C9400000C9400000C9400003C
:100010000C9400000C9400000C9400000C94000060
:100020000C9400000C9400000C9400000C94000050
:100030000C9400000C945C000C9400000C940000E4
:100040000C9400000C9400000C9400000C94000030
:100050000C9400000C9400000C9400000C94000020
:100060000C9400000C9400000FEF0DBF08E00EBFD1
:1000700010E02FEF27B90E943F007894FFCF0F9335
:100080001093800002E0009381001093820001E051
:1000900000936F001093000101E0009301010F91A4
:1000A00008950F930091010108B9000F06FD01E0CA
:1000B000009301010F9108950F93009100010395A2
:1000C000033019F40E9451000027009300010F91A2
:0200D000189581
:00000001FF
